:020000040800F2
:10000000B8090020DD020008491C00084B1C00084C
:100010004F1C0008531C0008571C0008000000007B
:100020000000000000000000000000005B1C000851
:100030005D1C0008000000005F1C00087B1C00081D
:10004000F7020008F7020008F7020008F7020008AC
:10005000F7020008F7020008F7020008F70200089C
:10006000F7020008D3150008F7020008F70200089D
:10007000F7020008F7020008F7020008F70200087C
:10008000F7020008F7020008F7020008F70200086C
:10009000F7020008F7020008F7020008EB15000855
:1000A000F7020008F7020008F7020008F70200084C
:1000B000F7020008F702000805050008F70200082B
:1000C000F7020008F7020008F7020008F70200082C
:1000D000F7020008290C0008F7020008F7020008E0
:1000E000F7020008F7020008F7020008DFF80CD05A
:1000F00004F04AFC00480047F51A0008B80900203F
:100100000CB50020019000906B48006840F48030EE
:100110006949086000BF6848006800F4003000903A
:100120000198401C0190009818B90198B0F5A06F93
:10013000F1D16148006800F4003010B10120009056
:1001400001E0002000900098012841D15B48006840
:1001500040F01000594908600846006820F003008C
:1001600008600846006840F0010008605248406896
:100170005149486008464068486008464068486001
:100180000846406820F47C1048600846406840F407
:10019000F81048600846006840F08070086000BFB2
:1001A0004548006800F000700028F9D042484068D7
:1001B00020F00300404948600846406840F00200D3
:1001C000486000BF3C48406800F00C000828F9D1A6
:1001D0000CBD10B5FFF794FF10BD10B53648006890
:1001E00040F001003449086008464068344908403E
:1001F0003149486008460068324908402E49086085
:100200000846006820F4802008600846406820F412
:10021000FE0048604FF41F008860FFF7DAFF4FF0E0
:1002200000602949086010BD10B50021002000229F
:10023000214B5B6803F00C0121B1042906D0082989
:1002400028D107E0214B224C236027E01F4B204C94
:10025000236023E0184B5B6803F47010164B5B6857
:1002600003F48032022303EB904022B9194B43433D
:10027000174C23600DE0104B5B6803F4003323B18F
:10028000144B4343124C236003E0104B4343104C88
:10029000236003E00D4B0E4C236000BF00BF064BF4
:1002A0005B68C3F303130C4CE15C094B1B68CB4048
:1002B000074C236010BD00000010024000200240E7
:1002C0000000FFF8FFFFF6FE08ED00E000127A00E4
:1002D0000000002000093D0004000020064880477F
:1002E00006480047FEE7FEE7FEE7FEE7FEE7FEE71B
:1002F000FEE7FEE7FEE7FEE7DB010008ED00000891
:1003000070B5044601F0BFFC054600BF01F0BBFC20
:10031000401B04EB4401C1EBC411B0EBC10FF5D39A
:1003200070BD70B5044601F0AEFC054600BF01F09B
:10033000AAFC401BA042FAD370BD000008B5684873
:10034000806940F00400664988610846806940F091
:10035000080088610846806940F001008861012139
:10036000084602F09DF901215E4801F0AEFF5E48AB
:1003700000685E4908405C490860084600685C49BE
:1003800008435949086058480830006840F4405014
:100390005549083108605748006857490840554991
:1003A00008600846006855490843524908605148AA
:1003B0000C30006840F0B0004E490C31086040201D
:1003C000ADF8000048208DF8030003208DF80200EE
:1003D0006946484801F0A8FE4348006820F47020B0
:1003E0004149086008460068454908433E4908609D
:1003F0003D480830006840F480503B4908310860AF
:100400000815ADF8000010208DF8030003208DF8CA
:1004100002006946374801F087FE4FF48061354895
:1004200001F02FFF8021334801F02DFF4FF4805160
:100430002D48001F01F027FF10212E4801F023FF57
:1004400020212C4801F01FFF08BD70B505460C4661
:10045000062D42D2DFE805F04103121E2A36012C98
:1004600005D121032048001F01F00BFF05E04FF4E8
:1004700080511D48001F01F006FF2EE0012C04D121
:1004800010211C4801F0FDFE03E01021194801F085
:10049000FAFE22E0012C04D12021164801F0F1FEE1
:1004A00003E02021134801F0EEFE16E0012C04D1F8
:1004B0004021104801F0E5FE03E040210D4801F025
:1004C000E2FE0AE024B180210A4801F0DAFE03E0EE
:1004D0008021084801F0D7FE00BF00BF70BD0000BA
:1004E000001002400004300004080140FFFFF0F05B
:1004F00000000303000C0140FFFF000F0000333039
:100500000000010110B501213C4803F026F8002845
:1005100037D03B480088401C80B2394908806428A5
:1005200004D1002008800120364908803648008820
:10053000401C80B234490880142804D1002008806F
:1005400001203249088032480088401C80B230497E
:1005500008800C2804D10020088001202D49088043
:100560002D480088401C80B22B4908800A2804D1FD
:100570000020088001202949088001211F4802F03D
:10058000FDFF10BD3EB505460C460121042002F0DA
:1005900094F81A4802F0E8F8A0B2ADF80400681E1A
:1005A00080B2ADF800000020ADF80600ADF8020002
:1005B0006946124802F0ACF90121104802F0CAFF66
:1005C000012211460D4802F01AFD01210B4802F0EC
:1005D000FBFC3EBD08B54FF4A06001F0D7FC1E2027
:1005E0008DF8000001208DF801008DF802008DF8D3
:1005F0000300684601F0CFFC08BD00000008004081
:10060000140000201C000020160000201E00002006
:1006100018000020200000201A00002022000020E6
:1006200070B505460C461021AD4801F02CFE284659
:1006300001F043FA0646204601F03FFA1021A8488F
:1006400001F01FFE304670BD70B504461021A4486D
:1006500001F019FE204601F030FA002001F02DFAD9
:10066000054610219E4801F00CFE284670BD2DE97C
:10067000F04107460D4616461021994801F003FE49
:10068000384601F01AFA8046002404E0285D01F0A3
:1006900014FA601CC4B2B442F8DB1021904801F097
:1006A000F0FD4046BDE8F0812DE9F04107460D46DA
:1006B000164610218A4801F0E6FD384601F0FDF9A2
:1006C0008046002405E0002001F0F7F92855601C61
:1006D000C4B2B442F7DB1021814801F0D2FD40469C
:1006E000BDE8F08170B504460D464FF400417C48EA
:1006F00001F0C9FD2A462146A020FFF7B8FF4FF4BC
:100700000041774801F0BDFD70BD70471FB575A170
:1007100003C9CDE9020100247448007908B9FFF744
:10072000F4FF052202A93020FFF7A1FF0522694648
:100730001020FFF7B9FF002408E01DF80400C228CC
:1007400002D0002004B010BD601CC4B2052CF4DB44
:100750000120F7E710B501F051F9FFF7D7FF10BD01
:1007600010B54FF400415E4801F08DFDFF21E220FD
:10077000FFF756FF05225E492A20FFF778FF012187
:100780002120FFF74DFF01212220FFF749FF2821FB
:100790002520FFF745FF20213120FFF741FF0F21E2
:1007A0002620FFF73DFF0F212020FFF739FF4FF4F0
:1007B00000414B4801F065FD10BD10B54FF40041FC
:1007C000474801F060FDFF21E120FFF729FF0522E6
:1007D00046493020FFF74BFF052244492A20FFF706
:1007E00046FF01212120FFF71BFF01212220FFF7F7
:1007F00017FF1A212420FFF713FF28212520FFF7D8
:100800000FFF0F212620FFF70BFF0E212020FFF7FF
:1008100007FF4FF40041324801F033FD10BD70B5C1
:1008200005464FF400412E4801F02DFD20222946B7
:10083000A020FFF71CFF4FF40041294801F021FDE3
:100840000720FFF701FF044621462720FFF7E8FEB7
:1008500004F0100028B1FF21E120FFF7E1FE102095
:1008600070BD04F0200008B12020F9E7FF20F7E771
:1008700010B50720FFF7E8FE044604F0400098B1E9
:100880001C480078401C1B49087020221A4961202E
:10089000FFF70AFF12221849184803F0B1FC21465D
:1008A0002720FFF7BDFE002410BD70B504460720C9
:1008B000FFF7CAFE054629462720FFF7B1FE05F0DF
:1008C000400050B1202221466120FFF7D0FEFF21D9
:1008D000E220FFF7A5FE002070BD0120FCE700002C
:1008E00000080140C2C2C2C2C200000024000020B1
:1008F000290000202E000020E40000208A000020B3
:1009000089488A4948608A48486070478748006932
:1009100040F080008549086170478448C16801F053
:10092000010008B10120704701F0040008B1022065
:10093000F9E701F0100008B10320F4E70020F2E726
:1009400070B5044600BFFFF7E8FF0546012D00D053
:1009500006E00120FFF7E5FC601E84B2002CF2D116
:1009600000BF04B9FF25284670BD70B505460024B8
:1009700045F6FF70FFF7E4FF0446C4B96B48006911
:1009800040F002006949086108464561006940F08D
:100990004000086145F6FF70FFF7D2FF0446012CC6
:1009A00005D06248006920F00200604908612046D5
:1009B00070BD70B505460E46FF20FFF7C1FF044627
:1009C00094B95A48006940F00100584908612E80E6
:1009D000FF20FFF7B5FF0446012C05D053480069FE
:1009E00020F0010051490861204670BD0146088889
:1009F00070472DE9F04105460E461746002407E0F2
:100A000036F814102846FFF7D4FFAD1C601C84B2E2
:100A1000BC42F5DBBDE8F08130B503460C46154617
:100A2000002207E01846FFF7E1FF24F812009B1CA4
:100A3000501C82B2AA42F5DB30BD2DE9F05F804642
:100A40008A461746B8F1006F02D33A48804501D371
:100A5000BDE8F09FFFF754FFA8F1006B4FEA9B251C
:100A6000CBF34809C9F50074A74200DC3C464DE0D1
:100A70004FF0006101EB85208A142F49FFF7CCFF6E
:100A800000260BE009EB06002B4931F810004FF669
:100A9000FF71884200D003E0701C86B2A642F1DBF1
:100AA00000BFA6421BDA4FF0006101EB8520FFF783
:100AB0005CFF002608E03AF8160006EB09011E4A22
:100AC00022F81100701C86B2A642F4DB4FF00061E0
:100AD00001EB85208A141849FFF78BFF04E02246BA
:100AE00051464046FFF785FFA74200D10FE06D1C3D
:100AF0004FF000090AEB440AA044381B87B2B7F54F
:100B0000007F02DD4FF4007400E03C46B0E700BF18
:100B1000FFF7FCFE00BF9BE713B50446012201A9C5
:100B20002046FFF78AFF1CBD2301674500200240D5
:100B3000AB89EFCD000001082401002008B5252075
:100B40008DF8000000208DF801008DF802000120D2
:100B50008DF80300684601F01EFA08BD2DE9F05F2C
:100B600005460E46300103F0B6FD8146FE4905FB01
:100B700001F003F0B0FD8246494603F0DDFB074675
:100B8000384603F0D7FD84B2204603F0A4FD834627
:100B9000394603F09CFB82464FF0834103F09AFBF9
:100BA000814603F0C7FD80464FF6FF7000EA04144B
:100BB00004EB080084B2ED48806940F00400EB4982
:100BC00088610846806940F480408861E848006890
:100BD00020F47F60E64908600846006840F40B6036
:100BE0000860E248C06840F48040E049C8600846B8
:100BF000C06820F48040C860DE480480001D008882
:100C000042F20C010843DB49091D088008460088B0
:100C100040F4807008800846008840F0200008807A
:100C2000FFF78CFFBDE8F09F10B540F22551D14889
:100C3000083802F067FEC8B140F22551CD480838A7
:100C400002F08AFECB48001F0088CB490968087073
:100C5000C9480068401CC849086008460068C74980
:100C6000401A802802D10846C349086010BD2DE90A
:100C7000FF410025C0490968C14A1268881A03F07B
:100C80002FFD21F0004106460022BE4B03F07AFD05
:100C900001D2BDE8FF8124E0ADB9B9480068007811
:100CA000242810D1B648006840784D280BD1B448AC
:100CB000006880783C2806D1B1480068C01CB04963
:100CC0000860012504E0AE480068401CAC4908609B
:100CD000AB480068A949401A802802DB0846A849A9
:100CE00008602DB9A6480068A34909688842D3D195
:100CF000002D6ED0A248006800780B286AD2DFE889
:100D000000F0D43853A3AF6A71BB8A06070000BF56
:100D10009B4800680078092806D19B48C08840F0AD
:100D200080009949C88005E09748C08820F080007D
:100D30009549C880002419E091480068401C9049FA
:100D40000860084600688D49401A802802DB084682
:100D50008B4908608A48006800784FF47A7101EB8B
:100D600080018948083020F81410641C042CE3DB4F
:100D70009CE08548807900F00100A0B98248C088D5
:100D800040F001008049C8800846C08820F08000FB
:100D9000C88040F2DC50088101467B484181818156
:100DA0004FF47A71C18181E07748807900F00100C9
:100DB00028B17548C08820F001007349C8804FF4FD
:100DC0007A707149088101466F4841818181C181F2
:100DD0006CE071E069E06C48C08840F008006A4946
:100DE000C88063E000240EE065480068401C644948
:100DF0000860084600686149401A802802DB0846FE
:100E00005F490860641C052CEEDB5D4800680078D3
:100E10005D4908744AE000240EE059480068401C0F
:100E200057490860084600685449401A802802DB88
:100E3000084653490860641C062CEEDB50480068E5
:100E400000785149487431E04F48807900F004003F
:100E500028B94D48C08840F004004B49C88025E0BF
:100E60004948807900F0040028B14748C08820F044
:100E700004004549C88019E000240EE0404800689D
:100E8000401C3F490860084600683C49401A8028D9
:100E900002DB08463A490860641C072CEEDB384840
:100EA000006800783849887400E000BF00BF34480B
:100EB0000068401C3249086034480078401C3349BF
:100EC00008700846007803286CD10020087030A311
:100ED000D3E901021968DB6801AE0DC60091304804
:100EE0008089000A8DF801002D48007B8DF80200F2
:100EF0002B48C089000A8DF803002948807B8DF8B3
:100F000004002748008A000A8DF805002448007C68
:100F10008DF806001C48C07C8DF807002048807AB8
:100F20008DF8080018490989A1F57A70C11700EBFE
:100F30009171C1F387018DF8091013494989A1F511
:100F40007A70C11700EB9171C1F387018DF80A1017
:100F50000D49C989A1F57A70C11700EB9171C1F3F0
:100F600087018DF80B101EE040420F000010024078
:100F7000040801400838014030000020240500200A
:100F800034000020000028407600002039000020B6
:100F9000FF0000000000000000000000006E0000E4
:100FA0008A00002021E048498989A1F57A70C1179B
:100FB00000EB9171C1F387018DF80C104348007963
:100FC0008DF80E0000240DE000F05DFE06461DF8D1
:100FD00004003F49088000BF00F055FE801B5028E8
:100FE000FAD3641C0F2CEFDB00BF00BF51E6704743
:100FF00010B538480078002841D0002035490870E5
:10100000112035490870FF2048708870C870087139
:10101000FFF7D3FB00F037FE81B22B48818100F04F
:1010200032FEC0F30F212848C181007B2A49087095
:1010300025488089001248702348807B88702248A8
:10104000C0890012C87008460078401C2349087007
:101050002148407848702048807888701E48C078C1
:10106000C87040F2DC501849088101461648418199
:1010700040201B4908701B49087000F074FF1A4893
:101080000078401C18490870184801780120FFF7C3
:10109000DCF9164801780220FFF7D7F913480178E8
:1010A0000320FFF7D2F910480078FF280AD10F4833
:1010B000007808B9012000E000200C4908700020E9
:1010C0000949087010BD0000760000208A00002049
:1010D00004380140380000202400002029000020AE
:1010E00046000020450000203B0000203A00002080
:1010F000E448806940F00400E2498861084680695C
:1011000040F008008861E04800686FF30B00DE499A
:101110000860DE48006820F00F00DC490860D9480C
:10112000806940F40070D74988610846C06840F47F
:101130000070C8600846C06820F40070C8600846A7
:10114000406820F4404048600846406840F4004051
:101150004860CF480068CF490840CD49086008463C
:10116000006808600846006820F480700860081D68
:10117000006820F00200091D08600846006820F49D
:10118000602008600846006840F460200860084657
:10119000006840F4801008600846006820F4006091
:1011A00008600846006840F400000860B84828302D
:1011B000006820F47000B6492831086008460068CD
:1011C00000200860B2480C30006820F03800B049B8
:1011D0000C3108600846006840F038000860081FBD
:1011E000006820F4E010091F08600846006840F419
:1011F000E0100860081F006840F00100091F086047
:101200000846006840F00800086000BFA048001DC4
:10121000006800F008000028F8D19D48001D006813
:1012200040F004009A49091D086000BF9848001D5D
:10123000006800F004000028F8D170470146944887
:101240003030006820F01F00914A303210601046A4
:101250000068084310608E48001D006840F480005C
:101260008B4A121D106000BF8948001F006800F003
:1012700002000028F8D086484830006880B27047E5
:1012800070B506460B460024002505E03046FFF702
:10129000D5FF0444681CC5B29D42F7DBB4FBF3F0F4
:1012A00080B270BD2DE9FE4F0024A14608E0102059
:1012B000FFF7C4FF204484B209F1010000F0FF09E8
:1012C000B9F1140FF3DB142094FBF0F084B2204644
:1012D00003F001FA824603F041FA07464FF0663206
:1012E0006D4B03F00EF9054603F07CFA029002986C
:1012F00003F034FA0546694A694B03F0FFF80746E4
:10130000684A694B03F06FF90022684BCDE9000190
:1013100003F050F8824603F065FA0290644902989F
:1013200002F0D8FF0290029803F0EBF9BDE8FE8FBF
:1013300010B56048007850BB4021544800F087FF4A
:1013400028B95D480078401C5B49087002E0002025
:101350005949087058480078962844DD00205649BD
:1013600008704FF48061494800F08DFF80214748A4
:1013700000F087FF4FF47A70FEF7C2FF4FF48061F0
:10138000424800F07EFF01204A4908702BE04021CE
:101390003E4800F05CFF30B1012048490870002051
:1013A000454908701FE045480078E0B142480078A0
:1013B000401C4149087008460078502813DD4FF45E
:1013C0008061324800F05FFF4FF49670FEF798FF9F
:1013D00080212E4800F057FF4FF480612B4800F029
:1013E00050FF00BFFEE710BD2DE9FE4F34480290CC
:1013F00005210820FFF744FF0190019803F070F9E0
:10140000804600222F4B03F0EEF806464FF0604274
:101410002D4B03F076F8044600224FF0804303F092
:1014200070F8824603F0DEF90090009803F096F918
:1014300004460022254B03F0A5F921D22448006878
:10144000401C23490860084600680A280ADD214834
:10145000007808B9012000E000201E490870002033
:101460001B4908601B480078012804D18102074805
:1014700000F009FF04E04FF48061044800F001FF30
:10148000BDE8FE8F0010024000080140000C014042
:1014900004240140FFFFF00066664A3FE17A14AE83
:1014A00047E1F63F22FDF675E09C713F00003940B0
:1014B000000020413C0000203D0000203E000020B4
:1014C000D7A350400000B0407A140A4000000C40FE
:1014D00040000020440000207FB501210D2001F0D4
:1014E000DFF809208DF8080005208DF8090000209C
:1014F0008DF80A0001208DF80B0002A800F04BFDCA
:1015000017208DF8080006208DF8090000208DF8BE
:101510000A0001208DF80B0002A800F03CFDF94CF8
:10152000E514ADF80C5048208DF80F0003208DF81D
:101530000E0003A9204600F0F7FD0220ADF80C00D4
:1015400048208DF80F0003208DF80E0003A92046D7
:1015500000F0EAFD0820ADF80C0048208DF80F00DF
:1015600003208DF80E0003A9204600F0DDFDA01534
:10157000ADF80C0048208DF80F0003208DF80E0008
:1015800003A9E14800F0D0FD0321012000F0E2FEB4
:101590000820009000208DF804000C208DF8050034
:1015A00001208DF80600684602F084FB0821002027
:1015B00000F0D0FEA015009000208DF804000C2053
:1015C0008DF8050001208DF80600684602F072FBD8
:1015D0007FBD10B5082002F0D3FB28B10120CB4914
:1015E0000870082002F0DDFB10BD10B54FF48070CC
:1015F00002F0C6FB28B10120C5490870000202F0C4
:10160000D0FB10BD10B50221BE4800F020FE98B9F5
:101610000120C0490870C0480078401CBE490870CD
:10162000084600780F2873DD0A2008704FF48061A7
:10163000B44800F028FE6BE0B6480078002864D07B
:10164000B5480078082860DD0020B24908704FF4E2
:101650008061AC4800F015FEB0484089B0F5C86F15
:1016600010DDAE480089B0F5C86F0BDDAB48C0880F
:1016700040F01000A949C8800846C08820F020002A
:10168000C88032E0A548807900F0100048B1012000
:10169000A3490870A148C08820F010009F49C88065
:1016A00023E09E48807900F0200058B19B48C08814
:1016B00020F020009949C8800846C08820F08000AA
:1016C000C88012E09548C08840F020009349C88047
:1016D00040F2DC5191484181084690490881014619
:1016E0008E4881814FF47A71C1818C48C08820F086
:1016F00001008A49C8800846C08820F00400C880DC
:101700000846C08820F04000C88000208249087048
:101710008248807900F0200020B98048807900F06C
:10172000100040B1002079490870794908707D495E
:1017300008707D4908704FF40061724800F087FD21
:1017400098B901207749087078480078401C77499B
:101750000870084600780A281FDD0A2008704FF438
:101760008061684800F08FFD17E06E48007888B10E
:101770006E48007808280DDD00206A490870674827
:10178000C08840F008006549C8804FF480615D481A
:1017900000F077FD0020654908704FF480515948EA
:1017A00000F055FD18B90120614908701BE0604840
:1017B0000078C0B100205E49087001205749C87404
:1017C0000846807900F0200068B90846807900F06A
:1017D000010040B157480078592804DA554800788C
:1017E000401C544908704FF40051464800F02FFD4A
:1017F00018B90120504908701BE04F480078C0B16B
:1018000000204D49087002204449C8740846807978
:1018100000F0200068B90846807900F0010040B16E
:1018200044480078272804DD42480078401E41499A
:1018300008704FF48041334800F009FD18B90120C9
:101840003E4908701BE03D480078C0B100203B498C
:10185000087003203149C8740846807900F02000E0
:1018600068B90846807900F0010040B1344800783A
:10187000592804DA32480078401C314908704FF486
:101880000041204800F0E3FC18B901202D49087000
:101890001BE02C480078C0B100202A4908700420C1
:1018A0001E49C8740846807900F0200068B90846CF
:1018B000807900F0010040B121480078272804DD3C
:1018C0001F480078401E1E4908704FF400710D48F3
:1018D00000F0BDFC18B90120134908703BE0124824
:1018E000007870B10020104908700C48807900F031
:1018F000400048B30948C08820F040000749C8802C
:1019000029E028E0000C01400008014048000020C8
:101910004A000020470000205100002076000020EF
:1019200038000020490000204F0000205200002015
:101930004B000020450000204C0000204D000020FE
:10194000460000204E000020FFE72848C08840F0F5
:1019500040002649C8802648007810B925480078FC
:1019600060B125480078401C23490870084600787B
:10197000032800DA10BD00201F4908701C480078B9
:10198000D0B100201A4908701848807900F0010091
:1019900030B11648C08820F001001449C8800BE01F
:1019A0001248C08940F20E61884205DA0F48C088AB
:1019B00040F001000D49C8800E480078A0B1002019
:1019C0000C4908700948807900F0040030B10748DC
:1019D000C08820F004000549C88005E00348C0889D
:1019E00040F004000149C88000BFC3E77600002032
:1019F000480000204A0000205000002000B587B0B9
:101A00000121042000F04CFE0121082000F048FED6
:101A10000121080300F044FEE020ADF8040001209D
:101A20008DF8060018208DF8070001A92F4800F056
:101A30007BFB4FF40040ADF8040001208DF8060058
:101A400010208DF8070001A9284800F06DFB102038
:101A5000ADF8040001208DF8060010208DF8070075
:101A600001A9224800F060FB1021204800F009FC89
:101A70000020ADF808004FF48270ADF80A00002095
:101A8000ADF80C00ADF80E00ADF810004FF400708A
:101A9000ADF812001020ADF814000020ADF81600CB
:101AA0000720ADF8180002A9114801F095FF0121A7
:101AB0000F4802F036F807B000BD10B5044600BF6D
:101AC00002210B4802F0B1F80028F9D0214608485D
:101AD00002F058F800BF0121054802F0A6F80028DE
:101AE000F9D0034802F050F8C0B210BD0008014020
:101AF00000300140092000F02AF900F0B1F8474811
:101B000000684FF47A72B0FBF2F1B1F1807F00D33C
:101B10001DE021F07F40401E4FF0E0225061501741
:101B20000F22002807DA13071D0E3D4B00F00F04AB
:101B3000241F1D5503E013071C0E3A4B1C5400BF15
:101B400000204FF0E02290610720106100BF4FF4A9
:101B5000E13135480078FFF701F800F0CBF8FEF7E7
:101B6000CFFE00F0EDF9FEF7E9FBFFF7C1FAFFF752
:101B7000B3FCFEF7EFFDFEF720FE4FF47A712A4822
:101B80000078FEF7FFFC02F05DF945E02748008889
:101B9000012806D1002025490880FFF733FDFFF713
:101BA00023FC2348008801281AD102F0CEFA2148EC
:101BB000807900F0100080B900201F4908701F488C
:101BC0000078012804D001201C490870FEF7C8FDE8
:101BD0000120FEF795FBFEF74BFE0020144908801C
:101BE0001748008820B1002015490880FFF7A0FBA6
:101BF0001448008880B11148007820B100200F49B6
:101C00000870FEF7DAFD0B48807900F0100008B18B
:101C1000FFF7EEF902F03EFAB8E7000000000020FE
:101C200018ED00E000E400E0600000201C0000204F
:101C30001E000020760000205400002053000020E9
:101C40002000002022000020704700BFFEE700BFF8
:101C5000FEE700BFFEE700BFFEE770477047704732
:101C600000B585B0684600F0AEFC1F490098B0FB97
:101C7000F1F01E49086005B000BD1D480068401C19
:101C80001B490860704700BF194801684FF0E02009
:101C90008269174800688142F6D11448006800EB59
:101CA0004003C3EBC010C2EBC000104B1B68B0FB7D
:101CB000F3F001EB4103C3EBC11300EBC30070472A
:101CC00030B50446FFF7DFFF054600BFFFF7DBFF37
:101CD000401B04EB4401C1EBC411B0EBC10FF5D3C1
:101CE00030BD03480068704740420F005800002094
:101CF0005C00002010B5FEF76DFCFEF71FFF10BD65
:101D0000002054490861C86014204861002088619F
:101D1000C8610846006840F0010008600846406855
:101D20004D4908404B494860084600684B49084007
:101D3000484908600846006820F48020086008468A
:101D4000406820F4FE00486000208860704701462B
:101D50004048006840F001003E4A106010460068AC
:101D600010601046006840F48020106000BF3948C1
:101D7000006800F002000028F9D036484268881E4A
:101D800042EA8040334A5060104640685060104636
:101D9000006840F08070106000BF2E48006800F0BE
:101DA00000700028F9D02B48406840F00200294A12
:101DB00050608806000E2A4A10701046007870475E
:101DC00000B502460023FFF79BFF2248006840F45D
:101DD00080302049086000BF1E480068400C002881
:101DE000FAD04FF480601B494860901EC2B208468A
:101DF000406840EA824048600846406840F48030CD
:101E000048601848006840F03200164908601148E0
:101E1000006840F080700F49086000BF0D480068FE
:101E2000400E0028FAD00B48406840F002000949F3
:101E3000486005E007484068C0F3870303F00303E8
:101E4000022BF7D1901CC006000E05490870084609
:101E5000007800BD001002400000FFF8FFFFF6FE12
:101E6000600000200020024010B502224149424893
:101E7000FEF7D2FD3F480088012800D110BD0020A8
:101E8000FCE710B502223B493B48FEF7D6FD10BDEA
:101E900010B50924620037493748FEF7BDFD10BD73
:101EA00010B50924620033493348FEF7C6FD10BD62
:101EB0003048007B314908702E48808900124870F4
:101EC0002C48807B88702B48C0890012C870084657
:101ED0000078401C2A4908702848407848702748F4
:101EE000807888702548C078C8702248007C2549D1
:101EF00008702048008A00122349087070470120AA
:101F00001C4908801D4800781C49497800EB0120D5
:101F100018498881194880781849C97800EB012050
:101F200081B21448C181184800781649097801EB3C
:101F30000020104908827047FF201049087170473F
:101F400010B5FFF791FF20B1FFF7A2FFFFF7B0FF39
:101F500008E0FFF7F1FFFFF7D2FF012005490880F5
:101F6000FFF79EFF10BD10B5FFF7C9FFFFF798FF01
:101F700010BD0000A405002000F00008240000208F
:101F8000290000204500002046000020314901437F
:101F9000314A1160704770B5002100230F22C478C8
:101FA00004B32D4C246804F4E064C4F5E064210A11
:101FB000C1F10403CA40447804FA03F18478144060
:101FC00021430901254C0678A155047804F01F052A
:101FD0000124AC4005786D11AD0005F1E025C5F890
:101FE000004109E0047804F01F050124AC401C4DB9
:101FF0000678761145F8264070BD1A4A0A40024319
:10200000154B1B1F1A60704739B1134A121D126815
:102010000243114B1B1D1A6006E00F4A121D126885
:1020200082430D4B1B1D1A607047042808D14FF0E6
:10203000E021096941F004014FF0E022116107E05D
:102040004FF0E021096921F004014FF0E022116115
:10205000704700000000FA050CED00E000E400E02D
:1020600080E100E080FFFF1F10B50446CC488442A9
:1020700008D10121042000F02DFB0021042000F0F4
:1020800029FB46E0C748844208D10121082000F01E
:1020900021FB0021082000F01DFB3AE0C2488442E9
:1020A00008D10121102000F015FB0021102000F0C4
:1020B00011FB2EE0BD48844208D10121202000F010
:1020C00009FB0021202000F005FB22E0B8488442F3
:1020D00008D10121402000F0FDFA0021402000F04D
:1020E000F9FA16E0B348844208D10121802000F0BB
:1020F000F1FA0021802000F0EDFA0AE0AE488442B7
:1021000007D10121801500F0E5FA0021A01500F0AB
:10211000E1FA10BD10B50121084600F0DBFA0021FC
:10212000012000F0D7FA10BD2DE9F041024600254C
:102130000026002000230024002791F803C00CF0A3
:102140000F0591F803C00CF0100CBCF1000F03D088
:1021500091F802C04CEA050591F800C0BCF1000FEF
:1021600031D0146800202BE04FF0010C0CFA00F382
:10217000B1F800C00CEA03069E4220D183004FF064
:102180000F0C0CFA03F7BC4305FA03FC4CEA0404F9
:1021900091F803C0BCF1280F06D14FF0010C0CFAE6
:1021A00000FCC2F814C00AE091F803C0BCF1480F6B
:1021B00005D14FF0010C0CFA00FCC2F810C0401C15
:1021C0000828D1D31460B1F800C0BCF1FF0F34DD92
:1021D000546800202EE000F1080C4FF0010808FAC6
:1021E0000CF3B1F800C00CEA03069E4221D1830033
:1021F0004FF00F0C0CFA03F7BC4305FA03FC4CEA52
:10220000040491F803C0BCF1280F05D100F1080CBB
:1022100008FA0CF8C2F8148091F803C0BCF1480F1A
:1022200007D100F1080C4FF0010808FA0CF8C2F8C9
:102230001080401C0828CED35460BDE8F0814FF6D2
:10224000FF710180022181700421C1707047024634
:10225000002093680B400BB1012000E00020704784
:102260000146886880B2704702460020D3680B4060
:102270000BB1012000E0002070470146C86880B221
:10228000704701617047416170470AB1016100E028
:1022900041617047C16070474FF480320A438261E8
:1022A0008161826182698269704702460020434BE6
:1022B00018684FF68073184040EA021008433F4BFD
:1022C000186070473E49C8617047F0B50A46002360
:1022D00000240021002500F00046B6F1004F02D195
:1022E000364EF16901E0354E7168C0F3034583B2A3
:1022F00000F44016B6F5401F08D121F070612F4E52
:10230000766826F070662D4F7E6012E000F480162D
:10231000B6F5801F06D1032606FA05F4A14341F065
:10232000706106E0460D360103FA06F6B14341F04E
:10233000706122B1460D360103FA06F6314300F012
:102340000046B6F1004F02D11C4EF16101E01B4E78
:102350007160F0BD30B500228B071C0F0F2303FA0C
:1023600004F2164B08338C1053F824309343134C6B
:1023700008348D1044F8253023468C1053F824304F
:102380008C07240F00FA04F423430C4C08348D10FE
:1023900044F8253030BD0A49DC3108607047000040
:1023A00000080140000C01400010014000140140F1
:1023B00000180140001C01400020014000000140C5
:1023C00000002042DF48006840F00100DD4908605D
:1023D00008464068DC490840DA4948600846006819
:1023E000DA490840D74908600846006820F4802090
:1023F00008600846406820F4FE0048604FF41F0063
:1024000088607047CF49096821F48031CD4A116056
:102410001146096821F480211160B0F5803F03D096
:10242000B0F5802F0ED106E0C649096841F480312D
:10243000C44A116007E0C349096841F4A021C14AB8
:10244000116000E000BF00BF704710B501460022D8
:10245000002300204A11012A02D1BA4C236806E069
:10246000022A02D1B74C236A01E0B64C636A01F03C
:102470001F02012494401C400CB1012000E0002008
:1024800010BD38B5002000900024002500BF312089
:10249000FFF7DBFF05460098401C00900098B0F560
:1024A000A06F01D0002DF2D03120FFF7CEFF08B190
:1024B000012400E00024204638BD01460020A14A46
:1024C000106820F0F80040EAC10010607047A04991
:1024D00008607047024600209A4B586820F47C1030
:1024E00042EA01031843974B5860704798490866C1
:1024F000704701460020934A506820F003000843CB
:10250000506070478F48406800F00C0070470146EB
:1025100000208C4A506820F0F0000843506070475B
:1025200001460020874A506820F4E060084350606C
:10253000704701460020834A506820F4605040EA0A
:10254000C1005060704729B17E4A527A02437D4BE8
:102550005A7204E07B4A527A82437A4B5A7270472D
:102560007B49D8310860704701460020754A5068A1
:1025700020F440400843506070470021714A2032E7
:102580001170704A82F82010012802D004280AD164
:1025900004E001216B4A2032117005E00521694AEF
:1025A0002032117000E000BF00BF70476949086029
:1025B00070476449096A0143624A1162704765497C
:1025C00044390860704730B5002100220024002300
:1025D0005C4D6D6805F00C0121B1042905D0082976
:1025E00023D105E05C4D056022E05B4D05601FE0F6
:1025F000544D6D6805F47012524D6D6805F48034C9
:10260000022505EB92421CB9544D554305600BE081
:102610004C4D6D6805F400351DB1504D55430560B6
:1026200002E04D4D5543056002E04B4D056000BF93
:1026300000BF444D6D6805F0F0010909484D6B5C21
:102640000568DD4045603F4D6D6805F4E061090AAD
:10265000434D6B5C4568DD4085603A4D6D6805F41F
:102660006051C90A3E4D6B5C4568DD40C560354D23
:102670006D6805F44041890B3A4D6B5CC568B5FB4C
:10268000F3F5056130BD29B12E4A526902432D4B45
:102690005A6104E02B4A526982432A4B5A617047BF
:1026A00029B1284A92690243264B9A6104E0254ADF
:1026B00092698243234B9A61704729B1214AD269BA
:1026C0000243204BDA6104E01E4AD26982431D4B6B
:1026D000DA61704729B11B4AD2680243194BDA60AC
:1026E00004E0184AD2688243164BDA60704729B179
:1026F000144A12690243134B1A6104E0114A126929
:102700008243104B1A617047124940390860704784
:102710000F49C86470470B49C87170470948406A3F
:1027200040F0807007494862704701460020054A22
:1027300092680A400AB1012000E000207047014978
:1027400088727047001002400000FFF8FFFFF6FE9D
:10275000000042428004424200127A0000093D001B
:10276000610000207100002010B50446FE4884423C
:1027700008D10121C014FFF7ADFF0021E014FFF7DD
:10278000A9FFC4E0B4F1804F08D101210846FFF74A
:10279000AEFF00210120FFF7AAFFB8E0F348844212
:1027A00008D101210220FFF7A2FF00210220FFF73C
:1027B0009EFFACE0EE48844208D101210420FFF7DF
:1027C00096FF00210420FFF792FFA0E0E948844231
:1027D00008D101210820FFF78AFF00210820FFF718
:1027E00086FF94E0E448844208D101211020FFF7DD
:1027F0007EFF00211020FFF77AFF88E0DF48844247
:1028000008D101212020FFF772FF00212020FFF7CF
:102810006EFF7CE0DA48844208D101214014FFF7C2
:1028200059FF00216014FFF755FF70E0D54884423E
:1028300009D10121C804FFF74DFF00214FF400200A
:10284000FFF748FF63E0D048844209D10121080521
:10285000FFF740FF00214FF48010FFF73BFF56E0E9
:10286000CA48844209D101214805FFF733FF0021FE
:102870004FF40010FFF72EFF49E0C548844208D10D
:1028800001214020FFF733FF00214020FFF72FFFF9
:102890003DE0C048844208D101218020FFF727FF96
:1028A00000218020FFF723FF31E0BB48844208D19C
:1028B00001218015FFF71BFF0021A015FFF717FF6F
:1028C00025E0B648844209D101210804FFF702FF40
:1028D00000214FF48030FFF7FDFE18E0B04884423D
:1028E00009D101214804FFF7F5FE00214FF4003023
:1028F000FFF7F0FE0BE0AB48844208D101218804C9
:10290000FFF7E8FE00214FF48020FFF7E3FE10BD43
:1029100000220288944B98420ED0994B98420BD0DB
:10292000B0F1804F08D0914B984205D0904B98421F
:1029300002D0904B984204D14FF68F731A404B88C7
:102940001A438D4B984207D08C4B984204D04FF6D7
:10295000FF431A40CB881A4302808B8883850B88FB
:102960000385814B98420BD0854B984208D08B4B06
:10297000984205D08A4B984202D08A4B984201D1A6
:102980000B7A038601238382704770B500240022EE
:102990000023058C4FF6FE7635400584028C838833
:1029A000048B4FF68F752C40B51E2C400D882C43A0
:1029B000751E2A400D892A434D882A436A4DA84234
:1029C0000BD06F4DA84208D0744DA84205D0744D6D
:1029D000A84202D0734DA84213D14FF6F7752A4092
:1029E0004D892A434FF6FB752A408D882A434FF6BE
:1029F000FF652B404FF6FF552B408D892B43CD892A
:102A00002B4383800483CD888586028470BD70B596
:102A1000002400220023058C4FF6EF763540058414
:102A2000028C8388048B48F6FF752C404FF6FF45D7
:102A30002C400D884FF6FF7606EA05252C434FF60D
:102A4000DF752A400D8906EA05152A434D8806EAF6
:102A500005152A43444DA84202D0494DA8421DD134
:102A60004FF67F752A404D894FF6FF7606EA051529
:102A70002A434FF6BF752A408D8806EA05152A437A
:102A80004FF6FF352B404FF2FF752B408D8906EA3C
:102A900085052B43CD8906EA85052B438380048376
:102AA000CD880587028470BD70B500240022002304
:102AB000058C4FF6FF6635400584028C8388848B35
:102AC0004FF68F752C404FF6FC752C400D882C432B
:102AD0004FF6FF552A400D894FF6FF7606EA052589
:102AE0002A434D8806EA05252A431F4DA84202D0F5
:102AF000234DA8421DD14FF2FF752A404D894FF654
:102B0000FF7606EA05252A434FF6FF352A408D88D1
:102B100006EA05252A434EF6FF752B404DF6FF7554
:102B20002B408D8906EA05152B43CD8906EA05154C
:102B30002B4383808483CD888587028470BD70B5E4
:102B4000002200230024058C4EF6FF7635400584D4
:102B5000038C8488828B48F6FF752A404FF6FF4528
:102B60002A400D8820E00000002C014000040040B5
:102B700000080040000C004000100040001400401D
:102B800000340140004C014000500140005401401D
:102B900000180040001C00400020004000400140A0
:102BA00000440140004801404FF6FF7606EA052543
:102BB0002A434DF6FF752B400D8906EA05352B4358
:102BC0004D8806EA05352B43FA4DA84202D0FA4D4E
:102BD000A84208D14BF6FF752C408D894FF6FF7641
:102BE00006EA85152C4384808283CD88A0F8405066
:102BF000038470BD828B4FF2FF331A408283828B35
:102C00004FF6FF7303EA01231A4382837047F0B53E
:102C10000C461546002200210026078C4EF6FF7C4C
:102C200007EA0C070784828B018C4FF6FF7707EACF
:102C3000043640F6FF473A404FF6FF7707EA05278C
:102C40003A434FF6FF7707EA03373A43D94FB84282
:102C50000ED0D94FB8420BD0B0F1804F08D0D74F2B
:102C6000B84205D0D64FB84202D0D64FB84206D1AE
:102C70004DF6FF77394046F48057394305E047F673
:102C8000FF57394044F48057394382830184F0BDB3
:102C9000828B4FF6F3731A408283828B0A438283BE
:102CA0007047F0B50C461546002200210026078C1F
:102CB0004FF6FF6C07EA0C070784828B018C4FF6F6
:102CC000FF7707EA04264FF60C773A404FF6FF7776
:102CD00007EA03172F433A43B64FB8420ED0B64F18
:102CE000B8420BD0B0F1804F08D0B44FB84205D0F5
:102CF000B34FB84202D0B34FB84206D14FF6FF5798
:102D0000394046F48077394305E04FF2FF573940A8
:102D100044F48077394382830184F0BD028B4FF203
:102D2000FF331A400283028B4FF6FF7303EA01233D
:102D30001A4302837047F0B50C4615460022002165
:102D40000026078C4FF6EF7C07EA0C070784028BFE
:102D5000018C4FF6FF7707EA041640F6FF473A402A
:102D60004FF6FF7707EA03373A434FF6FF7707EA54
:102D700005273A438F4FB8420ED08F4FB8420BD041
:102D8000B0F1804F08D08D4FB84205D08C4FB8427B
:102D900002D08C4FB84206D14FF6DF77394046F06B
:102DA0001007394305E04FF65F77394044F01007CC
:102DB000394302830184F0BD028B4FF6F3731A404E
:102DC0000283028B0A4302837047F0B50C46154616
:102DD00000220021068C4FF6FE773E400684028BCF
:102DE000018C4FF60C7632407E1C06EA03162E4309
:102DF0003243704EB0420ED06F4EB0420BD0B0F1A5
:102E0000804F08D06D4EB04205D06D4EB04202D01A
:102E10006C4EB04206D14FF6FD76314044F00106CB
:102E2000314305E04FF6F576314044F00106314379
:102E300002830184F0BD70B505460C465D488542AD
:102E40000ED05D4885420BD0B5F1804F08D05B486D
:102E5000854205D05A48854202D05A48854200D161
:102E600000E000BF208850B92389A28861882846E5
:102E7000FFF7ABFFE1882846FFF79EFF25E020889B
:102E800004280AD12389A28861882846FFF753FFC6
:102E9000E1882846FFF742FF17E0208808280AD17A
:102EA0002389A28861882846FFF7FBFEE18828462F
:102EB000FFF7EEFE09E02389A28861882846FFF724
:102EC000A6FEE1882846FFF795FE70BD2DE9F0418A
:102ED00005460C4600260127608808B9022600E056
:102EE0000026A088012801D1022700E001272088C0
:102EF000A0B92389A28861882846FFF766FFE18888
:102F00002846FFF759FF23893A4631462846FFF7FE
:102F100012FFE1882846FFF701FF13E02389A2880A
:102F200061882846FFF707FFE1882846FFF7F6FE8D
:102F300023893A4631462846FFF747FFE18828466D
:102F4000FFF73AFFBDE8F0810A884B881A438B8867
:102F50001A43CB881A430B891A434B891A438B892E
:102F60001A43A0F8442070474FF6FF71818000217A
:102F70000180C18041800172704700210180418041
:102F80008180C180018141818181C181704700219F
:102F900001804180012181800021C1800181704731
:102FA0000021018041808180C18001814181818136
:102FB00070470000002C0140003401400004004034
:102FC00000080040000C004021B1028842F00102DC
:102FD000028004E002884FF6FE731A4002807047B8
:102FE00031B1B0F8442042F40042A0F8442005E09A
:102FF000B0F84420C2F30E02A0F8442070471AB182
:1030000083890B43838102E083898B4383817047EB
:103010008182704741EA0203A0F8483070471AB134
:1030200083890B43838102E083898B4383817047CB
:1030300001894FF6F8721140018170470A4600215C
:1030400001894FF68F73194011430181704730B5E4
:1030500004460D4629462046FFF7F0FF208940F040
:103060000700208130BD2DE9F04104460D4616468B
:103070001F46602D06D13B46012231462046FFF710
:103080005AFE05E03B46012231462046FFF79DFEF1
:1030900029462046FFF7D2FF208940F00700208113
:1030A000BDE8F08130B50C4600210189C9B24FF668
:1030B000FF7505EA0325154325432943018130BDEA
:1030C0002DE9F04105460E46174698460024434632
:1030D0003A4631462846FFF7E5FF2C894FF6F8704F
:1030E000044044F007044FF68F70044044F070042D
:1030F0002C81BDE8F081F0B504460D4616461F460A
:103100003B46324629462046FFF7CCFF208940F453
:1031100080402081F0BD0185828270470A460021EF
:1031200001884FF68F731940114301807047F0B545
:103130000C4615461E460021002200230189028B01
:10314000038C4FF6F877394021434FF6FC473A405D
:1031500040F201173A434FF6DD773B404FF6FF77D9
:1031600007EA06172F433B43018102830384F0BD26
:103170000A460021018B4FF68F73194011430183DA
:1031800070470A460021018B48F6FF7319404FF63D
:10319000FF7303EA02231943018370470A460021A3
:1031A000818B4FF68F7319401143818370470A4614
:1031B0000021818B48F6FF7319404FF6FF7303EA35
:1031C000022319438183704721B1028842F08002B3
:1031D000028004E002884FF67F731A400280704735
:1031E00021B1828842F00402828004E082884FF696
:1031F000FB731A408280704721B1828842F0080236
:10320000828004E082884FF6F7731A40828070470C
:1032100021B1828842F00102828004E082884FF668
:10322000FE731A40828070470A460021018B4FF6D8
:10323000F77319401143018370470A460021018B3F
:103240004FF2FF7319404FF6FF7303EA022319434D
:10325000018370470A460021818B4FF6F7731940AE
:103260001143818370470A460021818B4FF2FF731F
:1032700019404FF6FF7303EA022319438183704715
:103280000A460021018B4FF6FB731940114301835D
:1032900070470A460021018B4FF6FF3319404FF665
:1032A000FF7303EA02231943018370470A46002192
:1032B000818B4FF6FB7319401143818370470A4697
:1032C0000021818B4FF6FF3319404FF6FF7303EA5D
:1032D00002231943818370470A460021018B4FF670
:1032E0007F7319401143018370470A460021018B07
:1032F000C1F30E014FF6FF7303EA02231943018362
:1033000070470A460021818B4FF67F7319401143A5
:10331000818370470A460021818BC1F30E014FF66D
:10332000FF7303EA02231943818370470A46002191
:10333000018C4FF6FD7319401143018470470A4612
:103340000021018C4FF6F773194011430184704737
:103350000A460021018C4FF6DF7319404FF6FF73C8
:1033600003EA02131943018470470A460021018CC5
:103370004FF67F7319404FF6FF7303EA02131943A8
:10338000018470470A460021018C4FF6FF53194013
:103390004FF6FF7303EA02231943018470470A467C
:1033A0000021018C4FF2FF7319404FF6FF7303EABF
:1033B00002231943018470470A460021018C4DF60F
:1033C000FF7319404FF6FF7303EA02331943018478
:1033D000704730B5002301248C40A3B2048C9C4379
:1033E0000484048C02FA01F5ADB22C43048430BD90
:1033F00030B5002304248C40A3B2048C9C43048485
:10340000048C02FA01F5ADB22C43048430BD70B5D2
:103410000346002000241846183001258D40ACB228
:103420001D8CA5431D8409B1082909D100EB610059
:10343000056825F0700505600568154305600EE018
:103440000D1FC5F34E052844056825F4E0450560C9
:1034500005684FF6FF7606EA02263543056070BD23
:1034600021B1028842F00202028004E002884FF695
:10347000FD731A400280704721B1028842F00402B5
:10348000028004E002884FF6FB731A400280704706
:1034900021B1828842F08002828004E082884FF667
:1034A0007F731A408280704702884FF6F7731A4084
:1034B000028002880A430280704782884FF68F7329
:1034C0001A40828082880A438280704702894FF6C0
:1034D000F8731A40028102890A4302817047028907
:1034E0004FF67F731A40028102890A4302817047B6
:1034F0008184704781857047818670470187704756
:1035000081877047A0F84010704702884FF6FF434C
:103510001A40028002880A43028070470146888E62
:1035200070470146088F70470146888F70470146F3
:10353000B1F8400070470146888C70470146088DFD
:10354000704702460020138A0B400BB1012000E0B7
:1035500000207047CA430282704730B502460020FF
:1035600000230024158A05EA0103958905EA010470
:1035700013B10CB1012000E0002030BDCA4302822B
:103580007047000010B50446FB48844209D1012170
:103590008803FFF79FF800214FF48040FFF79AF867
:1035A00032E0F648844209D101214804FFF79FF830
:1035B00000214FF40030FFF79AF825E0F0488442EC
:1035C00009D101218804FFF792F800214FF48020EF
:1035D000FFF78DF818E0EB48844209D10121C804B7
:1035E000FFF785F800214FF40020FFF780F80BE08B
:1035F000E548844208D101210805FFF778F8002149
:103600004FF48010FFF773F810BD2DE9F04786B036
:1036100005460E460024A24600BFA1460027B089F9
:1036200000B100BF2F462C8A4CF6FF700440F08892
:1036300004432C82AC894EF6F3100440B0883189E3
:103640000843718908430443AC81AC8A4FF6FF40BC
:103650000440B0890443AC8201A8FEF7B4FFC64819
:10366000874202D1DDF810A001E0DDF80CA0A889A6
:1036700000F4004040B10AEBCA0000EB0A103168C8
:103680004900B0FBF1F807E00AEBCA0000EB0A10B2
:1036900031688900B0FBF1F86420B8FBF0F0040158
:1036A0002009642101FB1089A88900F4004040B181
:1036B000322000EBC900B0FBF1F000F0070004433A
:1036C00008E0322000EB09106421B0FBF1F000F0BB
:1036D0000F0004432C8106B0BDE8F0874FF416516B
:1036E000016000218180C18001810C214181002184
:1036F0008181704710B502460020108A4FF2FF0307
:1037000018400B884C8823438C882343CC88234360
:103710001843108210BD0021018041808180C1804A
:10372000704721B1828942F40052828104E082898B
:103730004DF6FF731A4082817047F0B503460024AE
:1037400000260025002040F66A17B94200D100BFCC
:103750001846C1F3421401F01F06012707FA06F5C7
:10376000012C01D10C3004E0022C01D1103000E01A
:1037700014301AB107682F43076002E00768AF43AF
:103780000760F0BD1AB1838A0B43838202E0838A0B
:103790008B4383827047028A4FF6F0731A4002828D
:1037A000028A0A430282704782894FF2FF731A40ED
:1037B000828182890A438281704721B1828942F0E5
:1037C0000202828104E082894FF6FD731A408281F1
:1037D0007047028A4FF6DF731A400282028A0A4358
:1037E0000282704721B1028A42F48042028204E0E0
:1037F000028A4BF6FF731A4002827047C1F3080237
:103800008280704701468888C0F30800704781892C
:1038100041F0010181817047028BD2B20283028B99
:1038200042EA012202837047028B02F47F42028344
:10383000028B0A430283704721B1828A42F0200240
:10384000828204E0828A4FF6DF731A4082827047D8
:1038500021B1828A42F01002828204E0828A4FF60D
:10386000EF731A408282704721B1828A42F00802C7
:10387000828204E0828A4FF6F7731A408282704790
:1038800021B1828942F40042828103E08289C2F33D
:103890000E028281704721B1828A42F400628282E4
:1038A00004E0828A4FF2FF731A4082827047828A54
:1038B0004FF6FB731A408282828A0A4382827047E3
:1038C00021B1828A42F00202828204E0828A4FF6AB
:1038D000FD731A408282704702460020B1F5007FD6
:1038E00000D100BF13880B400BB1012000E0002085
:1038F000704701F40072B2F5007F00D100BFCA43E7
:103900000280704770B50246002400230025002085
:1039100040F66A16B14200D100BFC1F3421501F072
:103920001F03012606FA03F3012D02D196893340C5
:1039300006E0022D02D1168A334001E0968A334018
:103940000C12012606FA04F41688344013B10CB1A7
:10395000012000E0002070BD10B50022002340F6D9
:103960006A14A14200D100BF0A1201249440A3B2FC
:10397000DC43048010BD00000038014000440040DA
:1039800000480040004C00400050004010B5044684
:10399000BE48844208D101218014FEF79BFE00211D
:1039A000A014FEF797FE16E0B948844208D1012121
:1039B0000014FEF79CFE00212014FEF798FE0AE09A
:1039C000B448844207D10121C013FEF790FE0021C4
:1039D000E013FEF78CFE10BD10B50022028802F441
:1039E00041520B884C8823438C882343CC88234343
:1039F0000C8923434C8923438C892343CC8923435B
:103A00001A430280838B4FF2FF74234083830B8A17
:103A1000038210BD2DE9F04F85B005460C464FF0EE
:103A2000000902274FF000084FF0010B0026B246B4
:103A3000A88B4FF240010840A88302202884B5F8E3
:103A40001C90A068022801D100BF38E0A08810B9FE
:103A50004FF0010B01E04FF0020B8D48854200D181
:103A600000E000BF6846FEF7AEFDDDF800A0E0888C
:103A7000B0F5007F0AD14FEA1A2000EB8000400029
:103A8000A168B0FBF1F0401D86B20BE04FEA4B108D
:103A9000BAFBF0F000EB80004000A168B0FBF1F051
:103AA000401D86B20A20B6FBF0F606F00108A6EB30
:103AB0000800C0F34F074FF6FF7000EA0828022FF6
:103AC00001DBFF2F02DD02274FF00008E08840EA0B
:103AD000080038432884A088A189084361880843E6
:103AE0002188084340F4006040EA0909A5F81C90C9
:103AF00005B0BDE8F08F0021018041808180C18048
:103B0000018141818181C1810721018270470021AA
:103B1000018041808180C1800221816000218181FA
:103B2000704721B1028842F04002028004E002881E
:103B30004FF6BF731A400280704721B1828B42F466
:103B40008062828304E0828B4FF6FF331A408283C7
:103B5000704730B5002400230C110125A540ABB2FD
:103B60001AB185881D43858002E085889D43858044
:103B700030BD1AB183880B43838002E083888B4376
:103B800083807047818170470146888970474FF66E
:103B9000FF62914204D0028842F48072028004E005
:103BA00002884FF6FF631A400280704721B1828875
:103BB00042F00402828004E082884FF6FB731A40D0
:103BC0008280704702884FF2FF731A400280028899
:103BD0000A4302807047018841F480510180704798
:103BE00021B1028842F40052028004E002884DF6BE
:103BF000FF731A400280704702460020012901D05D
:103C0000108B00E0908A70470146088A7047B1F532
:103C1000804F04D1028842F48042028004E002888E
:103C20004BF6FF731A40028070470246002013894A
:103C30000B400BB1012000E000207047CA43028115
:103C40007047F0B50246002000240023002501F053
:103C50000F070126BE40B4B20B1101269E40B3B23D
:103C6000968806EA03051689264016B10DB1012093
:103C700000E00020F0BD10B5002201F00F04012388
:103C8000A3409AB2D343038110BD0000003001402D
:103C900000380040003C0040002044490860091DF5
:103CA0000860091D0860091D086041483F4914313A
:103CB0000860704700213D498279002A3AD00A46BF
:103CC000126803689A430B461A600A1D126803685B
:103CD0009A430B1D1A60027911440A6803681A435B
:103CE0000A60324A0832126803689A432F4B08333D
:103CF0001A601A1D126803689A432C4B0C331A6021
:103D00004279102A0ED11A1F126803681A43274BF2
:103D100008331A601A1D126803681A43234B0C33C8
:103D20001A600DE02149427911440A6803681A4378
:103D30000A6005E0027911440A6803689A430A6040
:103D400070470021016001710C21417100218171D6
:103D500070471649103109680143144A1032116046
:103D6000704701460020114A143212680A400AB115
:103D7000012000E0002070470C49143108607047B2
:103D8000014600200022094B1B6803EA0102074B91
:103D900014331B680B4013B10AB1012000E000206E
:103DA0007047024914310860704700000004014068
:103DB000FFFF0F002DE9FC5F04460D46AE4903C925
:103DC000CDE900014FF4C8790198281A494690FBC3
:103DD000F1F7384600F076FC0646208801998842C3
:103DE00015DD2188019A881A00F06CFC8346314663
:103DF00000F070FA8046208800F06DFC8246414653
:103E000000F010FA074600F095FC208018E02088AA
:103E10000099884214DA2188009A881A00F052FC2E
:103E20008346314600F056FA8046208800F053FC65
:103E30008246414600F0F6F9074600F07BFC208000
:103E4000BDE8FC9F70B50F210220FDF719FA4FF471
:103E50007A71484301EB2030A0F2DC5040F2DC5193
:103E600001EB600081B2854881810F210020FDF7C0
:103E700007FA4FF47A71484301EB2030A0F2DC508E
:103E800040F2DC5101EB60007C4908810F210320E6
:103E9000FDF7F6F94FF47A7148434900A1EB203061
:103EA00081B27648C1810F210120FDF7E9F94FF475
:103EB0007A71484301EB2030A0F2DC5040F2DC5133
:103EC00001EB600081B26D4841810146C989A1F2D0
:103ED000DC5000F005FC21F0004104460022684B54
:103EE00000F068FC02D26548C08901E040F2DC5075
:103EF0006249C8810846C089B0F5FA6F02DD4FF407
:103F0000FA6001E05D48C0895C49C8810846C08903
:103F1000404210F57A7F03DA0846C089404200E04B
:103F20005848404281B25548C18101468989A1F271
:103F3000DC5000F0D5FB21F0004104460022524B3A
:103F400000F038FC02D24D48808901E040F2DC509C
:103F50004A49888108468089B0F5FA6F02DD4FF43E
:103F6000FA6001E045488089444988810846808993
:103F7000404210F57A7F03DA08468089404200E02B
:103F80004048404281B23D48818101460989A1F201
:103F9000DC5000F0A5FB21F00041044600223A4B22
:103FA00000F008FC02D23548008901E040F2DC5004
:103FB000324908810846008940F23A71884201DDA1
:103FC000084601E02D4800892C49088108460089EF
:103FD00040422C499639884203DA284800894042F9
:103FE00001E0284896384042244908814989A1F2D5
:103FF000DC5000F075FB21F0004104460022224B0A
:1040000000F0D8FB02D21D48408901E040F2DC50AC
:104010001A4948810846408940F23A71884201DDD8
:10402000084601E0154840891449488108464089FE
:10403000404214499639884203DA10484089404288
:1040400001E010489638404281B20C484181008915
:104050000E4909784FF40072C2EBC10108440749C8
:104060000881084640890A490978C2EBC101084421
:1040700081B20248418170BDF049000876000020FD
:104080000000244018FCFFFF00003E4046000020D6
:104090004500002010B514225249534800F0B0F8F2
:1040A0005148FCF7BCFB5148807900F0080020B96A
:1040B0004C48807900F0080058B14A48C08820F088
:1040C00008004849C8804948C08820F0080047498E
:1040D000C8804448C07C00B3012045490870810273
:1040E0004448FEF7D0F844480078401C4249087024
:1040F000084600781E2802DC3C48007A68B100209F
:104100003D4908703749C874394908703B490880EF
:104110004FF480613748FEF7B4F83548007888B925
:1041200036480088401C3549088008460088B0F5AC
:10413000805F07D1FDF717FF00203049088001207C
:104140002B490870012010BD704710B525488079B3
:1041500000F0100000B110BD2248807900F001008D
:1041600020B101210320FCF770F903E000210320B6
:10417000FCF76BF91B48807900F0200030B1012179
:104180000846FCF762F9FCF772FD0AE00021012005
:10419000FCF75BF91348807900F0100008B9FFF7CD
:1041A00051FE1048807900F0040020B10121022066
:1041B000FCF74BF903E000210220FCF746F909481F
:1041C000807900F0400058B101210846FCF73DF924
:1041D00001210220FCF739F901210320FCF735F910
:1041E00000BFB8E776000020E40000208A0000202D
:1041F000A0000020000C01409C0000209E00002038
:1042000040EA01039B0703D009E008C9121F08C058
:10421000042AFAD203E011F8013B00F8013B521ED8
:10422000F9D27047F0B480EA0102D40F4200B2EB39
:10423000410F02D20246084611464A0042D0C30D41
:10424000DDB2C1F3C752AD1A202D35DAC1F3160124
:1042500041F4000204B15242C5F1200602FA06F10F
:104260002A411044B3EBD05F23D0C4B1012DA0EBA1
:10427000C35009DCF0BC4FF0004202EAC352DBB28B
:1042800000F5000000F0F4BA400000F1807000EB8F
:10429000C350A0F1807040EAD170490009E049089C
:1042A00041EAC071A0EBC35000F50000400800EBEC
:1042B000C350F0BC00F0D3BA6142012202EB4101CD
:1042C000001BF6E7F0BC704781F00041AAE780F0E0
:1042D0000040A7E780EA010210B502F00043400069
:1042E00022D04A001FD0010E01EB1261C0F356002C
:1042F000C2F3560240F4000042F40002A0FB022088
:1043000000047F39140400D0401C50EA124001D44C
:104310004000491EC2B20C0604EBD010401C4008FD
:10432000802A02D003E0002010BD20F00100002907
:1043300000DA0020184310BD30B480EA010202F018
:10434000004530F0004221F0004013D090B1C30D81
:10435000D40DC2F31601C0F31600E41A41F40001B3
:1043600040F400027D34914201D3641C00E0490016
:10437000002C02DA30BC002070474FF4000000230C
:10438000914201D3891A034340084FEA4101F7D112
:1043900051B1914202D14FF0004105E002D24FF0FD
:1043A000010101E06FF0010103EBC450284430BC6F
:1043B00000F055BA2DE9FE4F804681EA0300C00F98
:1043C0000C46009021F0004123F00045B8EB0200BC
:1043D000A94105D24046214690461C460B4602465E
:1043E00023F00040104347D0270DC7F30A00C3F362
:1043F0000A510290401A019040286BDAC3F313006F
:1044000040F4801B0098924620B10023D2EB030AAF
:1044100063EB0B0B01985946C0F14002504600F087
:10442000FDF906460D4650465946019A00F005FA38
:1044300010EB08006141002487EA115284EAE77317
:104440001A4340D0009A62B3019A012A4FEA0752F8
:1044500015DC001B61EB02014FF0004202EA07523B
:10446000CDE90042001C41F5801132462B4600F098
:104470003CFA03B0BDE8F08F40462146F9E7001B47
:1044800061EB0201001C41F5801300185B4120180C
:10449000A2F5001747EB030140EAD570B6196D414C
:1044A00011E06D084FEA360645EAC0754FEA07523B
:1044B000001B61EB0201001C41F5801149084FEA25
:1044C00030000019514132462B4603B0BDE8F04F91
:1044D00000F0FCB90098012240000023D0EB02025A
:1044E00063EBE073009821464FEAE074B8EB0000FC
:1044F00061EB0401E9E783F000435BE781F00041F1
:1045000058E72DE9FE4F81EA030404F0004421F04E
:10451000004100944FF0000B23F0004350EA0104E7
:104520005ED052EA03045BD0C3F30A54C1F30A55C8
:104530002C44A4F2F3340194A0FB0254C1F3130100
:1045400041F48011C3F3130343F4801301FB0244CD
:1045500000FB034E840A970A44EA815447EA8357D2
:10456000A4FB076802958D0A05FB07854FEA932C8B
:1045700004FB0C542705029D4FEA065847EA1637FC
:10458000B5EB08056EEB070C870E920E47EA811714
:1045900042EA8312A7FB0201B6EB0B0164EB0004B5
:1045A0002B0D43EA0C335E1844EB1C50DA4651469F
:1045B000E7FB0201C5F313044FEA0B3343EA14533C
:1045C0004FEA0432019C43EA0603A4F10C0402946E
:1045D000009CCDE900B400F088F903B0BDE8F08F8D
:1045E00000200146F9E72DE9F04D81EA030404F0CB
:1045F000004B21F0004514464FF0000A23F0004123
:1046000050EA050220D054EA01021DD0C5F30A5732
:104610000246C5F31303C1F31300C1F30A5640F475
:10462000801543F48013A7EB0608101BD64608F24A
:10463000FD3873EB050002D308F1010801E0921880
:104640005B41B8F1000F03DA00200146BDE8F08DB0
:1046500000204FF48011064684460EE0171B73EBD2
:10466000050705D3121B63EB050306434CEA010C57
:1046700049084FEA300092185B4150EA0107EDD13A
:1046800052EA030012D082EA040083EA05010843DB
:1046900005D0101BAB4106D20122002306E0002208
:1046A0004FF0004302E06FF0010253101AEB0600D6
:1046B0004CEB085110EB0A0041EB0B01BDE8F04D4B
:1046C00000F004B9C10F80EAE0700844CA079623DD
:1046D000002100F0CDB896230022114600F0C8B8A2
:1046E0000EB5C10F80EAE0700844CA07002140F20D
:1046F00033438DE80E000A460B4600F0F6F803B08F
:1047000000BD00F0004220F00040C10DC0F31600D3
:1047100040F400007F2901DA00207047962903DC6D
:10472000C1F19601C84001E096398840002AF4D0D2
:104730004042704720F00040C10DC0F3160040F425
:1047400000007F2901DA00207047962903DCC1F1BF
:104750009601C840704796398840704700F0004283
:1047600030F000400AD0C10D01F56071C0F31600B1
:1047700042EA0151C2084007114370470020014638
:104780007047000030B5041E71F1000404DB4FF0E7
:104790000044404264EB0101141E73F1000405DB88
:1047A0001C464FF00043524263EB04038B4208BFA8
:1047B000824230BD30B5041E71F1000404DB4FF0BD
:1047C0000044404264EB0101141E73F1000405DB58
:1047D0001C464FF00043524263EB0403994208BF6A
:1047E000904230BD01F0004330B421F0004150EA66
:1047F000010206D00A0DA2F56072C1F31301002A6E
:1048000002DC30BC00207047440F44EAC104C10000
:10481000E01830BC00EBC25000F021B8202A04DBC5
:10482000203A00FA02F1002070479140C2F12003C3
:1048300020FA03F3194390407047202A06DBCB1778
:10484000203A41FA02F043EAE07306E041FA02F34B
:10485000D040C2F120029140084319467047002918
:10486000A8BF7047401C490008BF20F001007047F6
:1048700010B4B0FA80FC00FA0CF050EA010404BF56
:1048800010BC704749B1CCF1200421FA04F411FAAC
:104890000CF118BF012121430843A3EB0C01CB1DF0
:1048A0004FEA00614FEA102042BF002010BC704761
:1048B00000EBC35010440029A4BF10BC7047401C3B
:1048C000490008BF20F0010010BC704710B5141E4D
:1048D00073F1000408DA401C41F1000192185B41B9
:1048E0001A4301D120F0010010BD2DE9F04D924690
:1048F0009B4611B1B1FA81F202E0B0FA80F22032A7
:104900009046FFF78BFF04460F4640EA0A0041EA53
:104910000B0153465A46084313D0114653EA01008F
:1049200019D0C8F14002504600F040F805460E4646
:10493000504659464246FFF771FF084305D0012013
:1049400004E020463946BDE8F08D0020054346EAE4
:10495000E0762C4337430A986305E40AA0EB08008D
:104960000022FD0A44EA47540A3002D500200146DD
:10497000E9E7010510196941DDE9084500196941B8
:10498000BDE8F04DA2E70000064C074D06E0E068E8
:1049900040F0010394E8070098471034AC42F6D386
:1049A000FBF7A8FBF8490008184A0008202A04DB96
:1049B000203A21FA02F00021704721FA02F3D04098
:1049C000C2F12002914008431946704702E008C82E
:1049D000121F08C1002AFAD170477047002001E079
:1049E00001C1121F002AFBD17047000064000000C3
:1049F0007805000040060000184A0008000000206A
:104A0000A4000000CC490008BC4A0008A400002013
:104A100014090000DC4900080051250200000000D4
:104A2000000000000102030406070809000000005E
:104A300000000000000000000000000011FFFFFF68
:104A4000FF12FFFFFFFF00002405002024050020C7
:104A500001000100000000000000000000404000D4
:104A60000000000000000000000000000000000046
:104A70000000000000000000000000000001020330
:104A80000401020304060708090204060800244D75
:104A90003C000E000000DC05DC05DC05E80300003E
:104AA000000031313100FF00000000000000000074
:0C4AB000000000000000000001000000F9
:04000005080002DD10
:00000001FF
